:020000020000FC
:1000000012C0189518951895189518951895189563
:100010001895189518951895189518951895189578
:10002000189518951895F8948FED8DBF8CE087BBC7
:100030008FEF88BB929A8A9A8B9887E089B988E17A
:100040008AB983995DC383E080936F00552742E1AD
:100050006CD181E08093620080E080936100C29A5D
:10006000C398F1D1C39A183030F1012F16FD08C0A2
:1000700017FD03C0FCD132D2F2CFF9D134D2EFCF89
:10008000107E103E21F4D4D1AFD1D7D1E8CF103CAF
:1000900039F4CED1D8D1612FD6D1712FB0D1DFCFE5
:1000A000103619F4B7D1C9D1DACF103419F4C0D150
:1000B000B8D1D5CF4EC0113091F4C198B99AC0983B
:1000C000B89A3AE01BD2B99830916200332309F410
:1000D000339514D2B19BFECFC09AB898C0CF1230DE
:1000E00019F4C198B99ABBCF133011F4B998B7CFAE
:1000F000143089F11530D9F4A6D1A12EA4D1B12E96
:10010000A2D1C12EA0D1D12E08EE6ED1E62EF72EAF
:100110006C21C61639F47D21D71621F4CE24C09463
:10012000DF24D09414E1E6D010E0E4D098CF16306C
:1001300021F489D11093600092CF173039F483D124
:10014000A12E81D1B12E14E0D5D089CF103009F481
:1001500086CFC29885CF77D1103019F417EC83D1B0
:100160007ECF113051F413E87ED104EE4FEF51E011
:100170003BD1172F78D1A8D072CF123009F047C0E9
:1001800062D1F12E55D1242F352F002411242224A1
:10019000332400E16CD1A7D101E0000E0027101E2E
:1001A000201E301E03E636D1C62ED72E839B18C0E4
:1001B0000F2D047021F4D316C20691F003C003166C
:1001C000120671F012E00F2D017079F40F2D0870F6
:1001D00001F314E048D11C2D46D11D2D44D1D9CFB7
:1001E00012E80F2D027009F01064E12E3CD16CD0A2
:1001F0000E2D007441F0102D36D1112D34D1122D59
:1002000032D1132D30D10E2D007819F228CF1330B2
:1002100071F468D058F008EEE7D00FD192E080E09A
:10022000590F481F3150B8F72150A8F718CF143094
:1002300011F509D110936F00143089F05527103053
:1002400011F44EE910C0113011F44EE40CC012301C
:1002500011F446E208C0133011F442E104C04091A9
:1002600070005091710061D0EED010936100EBD01E
:1002700010936200F4CE153029F4E5D018BB1FEFBF
:1002800017BBEDCE163089F42DD070F008ECDBD022
:10029000612FD9D0712FB3D092E080E0590F481F61
:1002A0003150A0F7215090F7DACE173061F4CBD05F
:1002B000BFD0409370005093710010916F001430C4
:1002C00009F433D0CCCE45CF43E6042FA3D0B5D02C
:1002D00043954836D0F304EE4FEF56E085D0162F05
:1002E000C2D00895A5D0AFD0212FADD0312F31503D
:1002F00020400895612F626011D008EC4A2D5B2DDB
:100300006C2D7D2D7CD0612F636008D03AE0F6D053
:10031000612F626003D0612F01D0089500EC4091FD
:10032000600053EF762F6BD00895A42EB52ECC2409
:10033000AA0CBB1CCC1CAA0CBB1CCC1C002437E098
:10034000A30EB01CC01C38E4932EE1D0A02CB12C1D
:10035000C22C0FE9302E14E2412E20E0522E36E05E
:1003600033D060926B000AE618E136E02DD063943A
:1003700060926A0005E31CE0222734E025D06092F9
:10038000690060926C0039E01FD060926D0033E02C
:100390001BD060926E00300E411E521E00E513EC21
:1003A00020E036E911D0609263007092640030E47E
:1003B0000BD0609265007092660030E205D06092CA
:1003C0006700709268000895932EA1D0001A110A58
:1003D000220A632C742C852C869477946794060CDF
:1003E000171C281CA4D0089542D0042F40D0052FFC
:1003F0003ED074D042D0602F40D0702F089537D0B7
:10040000042F35D0052F33D0062F31D0072F2FD012
:1004100065D008952CD06CD030D0602F2ED0702FA6
:10042000089525D0042F23D0052F21D061D0089521
:100430000AD0412F08D0512F0895162F14D0172F0E
:1004400012D00895929A8399FECF92988399FACF09
:100450005F9BFCCF1CB1929A839BFECF08955F9B5C
:10046000FECF1CB108955D9BFECF1CB9089588E0B6
:10047000001F09D08A95E1F7089588E01BD0001F7E
:100480008A95E1F70895D0906C00E0906D00F090AF
:100490006E00B89A20F0C098DA94F1F704C0C098C2
:1004A000DA94F1F7C09AEA94F1F7C09AFA94F1F766
:1004B000B8980895D0906900E0906A00F0906B00C1
:1004C0008894B89AC098DA94F1F7B898EA94F1F75A
:1004D000B0990894FA94F1F7C09A08958091630056
:1004E0009091640010C080916500909166000BC0EF
:1004F000809167009091680006C003D03150E8F702
:10050000089587E59EE081509040E8F70895002423
:100510001124222438E0990C18F40A0C1B1C2C1C02
:100520003A9521F0000C111C221CF5CF0895662489
:1005300077248824FF24F394330C441C551C28F0A2
:10054000031414042504B8F78894579447943794F7
:1005500003141404250420F00318140825086394D8
:0E056000FA9421F0660C771C881CEFCF0895EA
:1007000080EE8DBF12E455D01CE453D04ED0173587
:1007100089F0123541F0193419F015E14AD0F6CFBD
:1007200015E547D0F3CF41D0F12F3FD0E12F149101
:1007300040D0ECCFD0E0C1E638D01993C238E1F711
:10074000D0E0C1E60991F02FEE278894F795E79560
:100750008894F795E7958894F795E7958894F795A9
:10076000E79503D016E025D0D1CF83E016D081E104
:1007700014D070E20990199081E00FD03296725037
:10078000C9F7E052F04085E008D081E106D067B7B4
:1007900066FF089581E101D0FACF67B760FDFDCF14
:1007A0006FB787BFE8956FBF08955F9BFECF1CB101
:0A07B00008955D9BFECF1CB908956B
:00000001FF
